:020000040000FA
:100000002F282034503475346C34733461346434A4
:100010006F34723465347334203470346134723424
:100020006134203463346F346E3463347534723425
:1000300073346F3473342034743465346C34653401
:10004000763469347334693476346F3473342034DD
:1000500031343634663436343234383441348316ED
:1000600085168617061786160616861506150516B2
:1000700005138513051085100511851106108610CE
:100080008113831207309F006A206400851E572861
:10009000861F5928061F5B28861E5D28061E5F28BE
:1000A000861D6128061D6328051E6528452805173D
:1000B000672885176728051467288514672805159C
:1000C0006728851567280614672886146728732013
:1000D0006A20452805138513051085100511851123
:1000E0000610861008002B30A000E230A100CD30B1
:1000F000A20064006400A20B7928A10B7728A00B52
:06010000752864000800F0
:02400E00143F5D
:00000001FF
